:0470000075C0FE2237
:007000018F
:0471000075C0FC2238
:0472000075C0F8223B
:0473000075C0F02242
:0474000075C0E02251
:0475000075C0C02270
:03000000020100FA
:03000B00021C6074
:03002300020317BE
:03002B000205EFDC
:030033000205DCE7
:03004300020B02AB
:03004B00020AEBBB
:10010000758180C2AFE4F5F8F5C8F5A875C0C312D3
:1001100001AA740012020275C0FF120C8074411211
:100120000C9C121C9DD2C8D2C9C2CCD2CBD2CDD28B
:10013000A9D2AF7433C0E07401C0E03016031214CA
:100140009D201303020C971206B130130C120A04FF
:100150001205B112043112015A221201A9C0E07431
:100160000E1214ACE563121C22D0E0C0E07436120B
:1001700014ACE558121C22D0E074121214AC900199
:100180009D2009169001A0E5F3B4060EE5F2B40037
:10019000099001A330C6039001A60214AF54580081
:1001A0005258004344002020002290F03CE493F891
:1001B000A3E493F5828883740212F020A3740212E0
:1001C000F020A374A212F02090F03FE493F8A3E48F
:1001D00093F5828883740212F020A3740212F02037
:1001E000A3744F12F0202260185389F0438901C292
:1001F0008DC28C854B8C854A8AD28C308DFDD5E0A2
:10020000EE2212F0351202092212024175670075C2
:1002100068B47565007566B4756900756A00D215B5
:10022000756D00756EA4756B00756CA4756F0075A7
:10023000700012023622E599C298C299D215D2AC4A
:1002400022C2ACE599C298C299D21522C2AC22C092
:10025000D0C082C083E570456F603F856E83856D39
:1002600082E0C0E0C082C083856E83856D82A385F5
:10027000836E85826DD083D082E56EB4B406756DD1
:1002800000756EA4C2ACE56F70021570156FD2AC2C
:10029000D0E0D083D082D0D0C322D083D082D0D03F
:1002A000D322C082C083C0E0C000C2ACF8E56AB40B
:1002B0001007E569B400028050856683856582E891
:1002C000F0C082C083856683856582A38583668549
:1002D0008265D083D082E566B4C406756500756614
:1002E000B4C082C083856A83856982A385836A8559
:1002F0008269D083D082301502D299D2C1D2ACD0DB
:1003000000D0E0D083D082C322C2C1D2ACD000D012
:10031000E0D083D082D322C0D0C082C083C0E0307E
:100320009941E56A45697006C299D215803585689C
:1003300083856782E0F599C299C082C0838568830E
:10034000856782A3858368858267D083D082E568CC
:10035000B4C4067567007568B4C215E56970021506
:100360006A156930984CE570B41007E56FB4000267
:10037000803E856C83856B82E599F0C082C0838561
:100380006C83856B82A385836C85826BD083D082DE
:10039000E56CB4B406756B00756CA4C082C083852F
:1003A0007083856F82A385837085826FD083D082AE
:1003B000C298D0E0D083D082D0D0327594007584BA
:1003C0008575879C75A408C2E8D294D29375D5FF31
:1003D00075E5FF12F0321203DCD2D822854D4F852D
:1003E0004C4EE54E2402F54EE54F3400F54F854F57
:1003F000D3854ED275B2F475B30075F20075F3066D
:10040000759369D2E94387102275500075510475C0
:100410005200755304754C00754D04754E00754FB0
:1004200004755600755700755400755500755800D1
:1004300022E558601B120451855383855282121A9B
:10044000391204874007C2C3120546D2C31204FE04
:1004500022C082C083855183855082E0F554A3E099
:10046000F555D083D082E555455470087550007518
:10047000510480DD855153855052E5522402F552D6
:10048000E5533400F55322200770AB55AA54E571AB
:007100018E
:100490002AFAEB3400FBEB30E76285538385528206
:1004A00078407901E82407F8E93400F97406121558
:1004B000D94049855383855282E582240DF582E532
:1004C000833400F583E020E013E5822407F582E51C
:1004D000833400F583E030E72330E0ED85538385F6
:1004E000528212186CB403148553838552821219F8
:1004F000C1B4CC02800280048000C322D322C08217
:10050000C083855183855082E0F8A3E0F9D083D081
:1005100082855153855052E552C398F552E553995F
:10052000F553E5522402F552E5533400F553C2C8A1
:10053000E55628F556E55739F557D2C88553518504
:1005400052501558D32220070F85538385528212AB
:100550001A0085835385825274C012F03B30070520
:10056000740012F03B120589C082C08385558385D3
:100570005482A3858355858254D083D082E5554526
:100580005470E274C012F03B22855383855282E09E
:10059000A3858353858252B4C00A74DB12F03B7486
:1005A000DC02F03BB4DB0774DB12F03B74DD02F0DD
:1005B0003BA2C692C2E557B44A02800E500C743A70
:1005C0001214AC9005D91214AF22743A1214AC90E4
:1005D00005D61214AF22524600202000C0D0C0829F
:1005E000C083C0E071DCD0E0D083D082D0D032C0F4
:1005F000D0C082C083C0E07549023013E7E557B42C
:100600004A0280E050DEE5F224FFF5F2E5F334F92A
:10061000F5F3C082C083854D83854C82E5F2F0A35B
:10062000E5F3F0D083D082E54C2402F54CE54D345F
:1006300000F54DE54CC395F2F54CE54D95F3F54DC0
:10064000E556C395F2F556E55795F3F557E54DB4E4
:100650004E028002402175F20075F300C082C08313
:10066000854D83854C82E5F2F0A3E5F3F0D083D08D
:1006700082754C00754D04055871DCD0E0D083D0F4
:1006800082D0D032755D00755E54755F0075605420
:10069000755900755A54755B00755C547561007529
:1006A0006200756300C2061206ECC209C20AC2D912
:1006B0002212F03E4017C2C11209E220D22E40F1B0
:1006C00012079C20D20840E912090980E422C213D3
:1006D00075C0FFC20775370012148774001214AC7E
:1006E0009012CB1214AF740012132E22D2C1C20387
:1006F000753700100673A95CA85BE8C39559F8E943
:10070000955AF9E948606220070AB90007B814024F
:1007100080024055E563B46302804EC082C0838589
:100720005A83855982E55BF0A3E55CF0D083D082E3
:10073000855C5A855B59C2CBE5612500F561E562B0
:100740003501F5620563D2CBE55AB49E02800240C2
:1007500018C082C083855A83855982E4F0A3F0D003
:1007600083D082755900755A54855A5C85595BE56A
:100770005B2402F55BE55C3400F55C20071A900110
:1007800040A95CA85BAA717B0012F02CE55B257187
:10079000F55BE55C3400F55CD205C322A82AB800FD
:1007A000081207B020D2084006752A14C3C2D2220C
:1007B000C0E0C000F874DDC0E07407C0E0E8A8291C
:1007C000B8001F752800752901B4410280147529ED
:1007D00005B42B02800C752900C2D2C322D000D0F0
:1007E000E022C0E0758309852982E52893F8D0E0EE
:1007F000B500150528E528B4030A752900752800F9
:10080000D2D2D322C2D2D322A8287900C0E0E99361
:10081000C000C001C082C083120909D083D082D039
:1008200001D00009D8E8D0E0752900752800C3C2BE
:02083000D222D2
:10090100415448002B2B2B00100545120995400836
:1009110012091A400302096522C0E0C000C001208B
:100921000624A95CA85BE8C39559F8E9955AF9E84A
:10093100C39402F8E99406F9E948600AC206D001B5
:10094100D000D0E0C322D206D001D000D0E0D32223
:10095100300708F537B4FF02807C22C0E074CC1266
:10096100097CD0E0C082C083855C83855B82F0A373
:1009710085835C85825BD083D08222855A838559A9
:1009810082C0E0E571042582F582E5833400F583B8
:10099100D0E0F022300748A837B800028041B80102
:1009A10002801BB80202801AB803028019B804023F
:1009B1008018B806028017B8FF028016801FF53331
:1009C100801BF5348017F5358013F536800FF5322D
:007200018D
:1009D100800B15811581158115810206CED322C3A5
:1009E10022B4C003D2D222100309B4DB12D203C253
:1009F100D2D322B4DC0474C08005B4DD0274DBC23E
:100A0100D2C3220531200A1720091BE56360173084
:100A1100C614120A28400FC2C0120A43020A6CE52A
:100A21006370F9020A5022901CF9E53193F8E5341C
:100A3100543FB5000280095007E5351201E7D32282
:100A4100C322C2E95387EFC2C7E5331201E722206F
:100A510090D4E5361201E712F0321203DC4387101D
:100A6100C2EBD2C7D2C0C209C20A22C20AD20975D8
:100A7100A408C082C083855E83855D82E0F55FA3A3
:100A8100E0F560D083D082E560455F7008755D0058
:100A9100755E5480DD8560E3855FE2E5E2C3955DC7
:100AA100F5E2E5E3955EF5E3E5E2C39402F5E2E5FF
:100AB100E39400F5E3855E83855D82E5822402F59A
:100AC10082E5833400F583121A39855EA3855DA220
:100AD100E5A22402F5A2E5A33400F5A375C285754C
:100AE100C300C2DBD2D975929922C0D0C082C08323
:100AF100C0E0D20AC2DBD2D9D0E0D083D082D0D03C
:100B010032C0D0C082C083C0E0C000C001D20AA9F7
:100B110060A85FE8C3955DF8E9955EF9E561C39565
:100B210000F561E5629501F562156385605E855F9B
:100B31005DC2DBD2D9201702D2C4D001D000D0E0EF
:070B4100D083D082D0D03236
:100C8000752F00753002120C8C021243900200E4A2
:100C9000F00582B582FA2212F03E400E12F0A11247
:100CA0000CB2120CC44003120D6922300B0312F077
:100CB0003B22C082C083853083852F82F0052FD0F0
:100CC00083D08222200F1891AB201007B4410ED29E
:100CD00010800AB42F02805BB4544DD20FD322206F
:100CE000E71BB53E028018B53C028021B53D02806D
:100CF0001CB4210280024005120D5291ABD322F5A3
:100D0000F0E52B6006152BE5F091ABD322301108EE
:100D1000C211B53D11020D3AB53C0BD211747FB52D
:100D20003D0280024014D322C20FC210C211752BA3
:100D300000D322121320B128C322900000E52B25F6
:100D400082F582E5833400F583E4F0121320B128A4
:100D5000C322C0E0900000E52B052B2582F582E53B
:100D6000833400F583D0E0F02274E3C0E0740DC05A
:100D7000E0752DFE752B00752C00900000E52B25ED
:100D800082F582E5833400F583E070057400021378
:100D90002E752E00052D052D900DEDE52D93FBA351
:100DA000E52D93FAEB4A7005740402132E8B838AA7
:100DB00082E52E052E93F9600B1212E6700122B522
:100DC00001B580E974D8C0E0740DC0E08B838A82DD
:100DD000E493A3B401FAE473E52B252CF52B752DD0
:100DE000FE8094752B00C20FC210C211220F930E09
:100DF000390EDB0EDE0F2D0FBF0F520FF90F360F1E
:100E0000770F6C113C113F0F49115B1164116E118A
:100E100071117F1185119411990FC50FCA11A60F79
:100E20004011FF12400F960F9A0FA60F9C0F9E0FB6
:100E3000980FA00FA30FA600004300011212E6B402
:100E40003F02805E152CC082C083C000C0019000AC
:100E500000E52B252C2582F582E5833400F583A956
:100E600083A8827A107B01121CB04024900000E518
:100E70002B252C2582F582E5833400F583E060057F
:100E8000052CB42CE77400D001D000D083D082228E
:100E9000740412132ED001D000D083D08215811596
:100EA0008122900140780079017A107B011219208B
:100EB000900ED112F05C90010012F05F121320909E
:100EC0000ED612F05C90011012F05F12132074FF26
:100ED000225352433A004453543A0044540044507D
:100EE0000001C082C083C000C001900000E52B2536
:100EF0002C2582F582E5833400F583AB83AA8278C2
:100F0000007901121CB04013C2C5D2137400121430
:100F1000AC9012D31214AFE5388002740412132E71
:100F2000D001D000D083D0821581158122450001E7
:100F30001211EC920B22264400011211EC921222A3
:100F40005600011211EC920D225100011211EC9287
:100F50000C22404B0001D207C2C5D21374001214F8
:100F6000AC9012D31214AF1581158122264C340097
:100F7000011211EC921722264C434400011211EC8D
:100F80009216500E12148474001214AC9012CB12EC
:100F900014AF2241540042004C004D00580059004B
:100FA000265000265700265900011212E6C394303D
:007300018C
:100FB000B40A0280024005152C74042274002248F1
:100FC0000001D2C5222654553D0026545500011279
:100FD00012E690FC6EB43102801690FFACB432027F
:100FE000800E90DC08B430028006740412132E22A6
:100FF00085834B85824A7400224900011212E690D3
:101000001114B431028026901105B43302801EB44D
:1010100034028022B435028035B43602805A9010F2
:10102000F4B430028007B432028002152C12F05C56
:1010300012132074FF2290111412F05C121320740A
:10104000FF2212F05C12F04D12132074FF22901157
:1010500019854BF0854AE0114275F000901120E5AA
:10106000331142901127E534114290112EE53511CC
:1010700042901135E53680CAC082C083C001C002EB
:10108000853083852F827A101210C61210A2121397
:1010900020E5822410F582DAEFD002D001D083D08F
:1010A0008222C082C083742012F03B7910E0058256
:1010B00012F053B90904742D8002742012F03BD948
:1010C000ECD083D08222C082C083742712F03B7997
:1010D00010B90805742D12F03BE00582B41F0280A0
:1010E000045002742E12F03BD9E7742712F03BD063
:1010F00083D082224D434231353220534C49502F08
:101100004158323500534C49502076332E3020312F
:10111000393939002D2D2D2D00756E6974733A0003
:1011200064656C61793A0070657273743A00736C2F
:101130006F74203A007461696C203A00444C004F8F
:101140000001C2C5D21374001214AC9012D3121451
:10115000AFE53812132E15811581222654584445C7
:101160004C4159002654584400017833805526508C
:101170000026504552534953540001783480442688
:10118000534C4F540026534C4F5454494D45000185
:101190007835802F26545854002654585441494CD1
:1011A00000017836801D5300011213044012B9006B
:1011B0000FE8B40A0280024002740A2439F880035E
:1011C0007404221212E6B43D028010B43F02800281
:1011D0008017E612F04A121320800BAA00121304A3
:1011E0004007E8A802F674FF227404221212E6B443
:1011F00030028007B431028004152CC322D322268A
:101200004300011212E6B43F02802A7801B4300292
:1012100080207805B431028019780AB43202801235
:10122000780BB43302800B780CB43402800478015C
:10123000152C883822E53812132E12132074FF2241
:101240005A00011203BB120409120684752B0075A3
:101250002A14C20FC210C211C217C20CD20DD20B77
:10126000D212C207C208753900753A00753B2B755A
:101270003C0D753D80753E08753F0275401E7541F9
:101280000275420675430E753801754A08754BDCC8
:1012900075330F75343F7535077536017537009016
:1012A00012DB780079017A087B0012F0269012E2B6
:1012B000781079017A087B0012F026780079017A9B
:1012C000107B01121CB0C213C216224F46464C4975
:1012D0004E450020202020202020004D4342313563
:1012E000320051535400C082C083900000E52B258A
:1012F0002C052C2582F582E5833400F583E0D0832C
:10130000D082C3227800790051E6600C12F0AA4026
:101310000712F0B0400680F0152CC322152CD32202
:10132000E53C12F03BE53D20E70312F03B22200CA8
:101330003C200D0812F04A712002136DB4FF0280A8
:101340002CB41C02800250212390136E2582F5825A
:10135000E5833400F583E493C0E0740193F582D013
:101360008312F05C712002136D741E712E2213AE75
:1013700013B113B913BE13C913CF13DC13E913EE62
:10138000148213F814051412141F14821482148288
:1013900014821482142D1482143B14821482144972
:1013A000148214571482146513AE147300004F4B4B
:1013B00000434F4E4E4543540052494E47004E4F56
:1013C0002043415252494552004552524F52004328
:1013D0004F4E4E4543542031323030004E4F204462
:1013E00049414C20544F4E450042555359004E4FF1
:1013F00020414E5357455200434F4E4E45435420D3
:007400018B
:101400003234303000434F4E4E4543542034383050
:101410003000434F4E4E4543542039363030004360
:101420004F4E4E45435420313434303000434F4EFC
:101430004E45435420313932303000434F4E4E45F3
:10144000435420323136303000434F4E4E454354E2
:1014500020323430303000434F4E4E45435420321A
:101460003634303000434F4E4E45435420323838E6
:10147000303000494E5445524E414C204552524F57
:1014800052002000121516C082C08390C400742040
:10149000F005827480B582F6D083D08222C082C0EB
:1014A0008390C4001214F4D083D08222F56422C049
:1014B00082C083C000C001C0E0C0A079C4A8648914
:1014C000A0E493600B547FF2A308B800F40980EF06
:1014D0008864D0A0D0E0D001D000D083D082C322D5
:1014E000C082C0837583C4856482547FF00564D054
:1014F00083D08222C082C083C0E0C00078507402D2
:10150000121547E4E0A3C2E7121557D8F6D000D071
:10151000E0D083D08222C0007803740312157B745C
:101520000512F014D8F4740212157B7420121547BA
:1015300074011215477406121547740C121547747E
:101540000212F014D00022C0E0C4540FB17BD0E0EE
:10155000540FB17BB16B22C0E0C4540F4440B17B47
:10156000D0E0540F4440B17BB16B22C0E075A1AF15
:10157000E5A120E3FB75A120D0E0224480F5A15431
:101580007FF5A122C082C083C000C001C0027406E2
:101590001215D94038E5822406F582E5833400F53A
:1015A00083E82406F8E93400F9E0541FFA89A0E240
:1015B000541FB50218A3C082C08389838882A3A95F
:1015C00083A882D083D08230E0C4C38001D3D0020C
:1015D000D001D000D083D08222C082C083C000C09E
:1015E00001C002C007C3601DFFE0FA89A0E2B50296
:1015F00017C082C08389838882A3A983A882D083ED
:10160000D082A3DFE4C38001D3D007D002D001D0C1
:1016100000D083D08222C082C083C000C001C0023B
:10162000C0037A06E0A320E02703B42002803BB485
:101630005B0280195017B4300280024010B441029E
:101640008011500FB43A0280024008800002170B4C
:1016500002170F89A0F2C082C08389838882A3A960
:1016600083A882D083D082DABB0A1AEA2582F58267
:10167000E5833400F583E0FB541E036054C0E08929
:10168000A0742DF2C082C08389838882A3A983A815
:1016900082D083D082D0E0B40A028002401DC3947D
:1016A0000AC0E0743189A0F2C082C0838983888235
:1016B000A3A983A882D083D082D0E0243089A0F26D
:1016C000C082C08389838882A3A983A882D083D063
:1016D00082EB20E01BE489A0F2C082C0838983886A
:1016E00082A3A983A882D083D0827400C302171674
:1016F000E489A0F2C082C08389838882A3A983A8D9
:1017000082D083D0827401C302171674FD800474E2
:10171000FF8000D38000D003D002D001D000D0835E
:10172000D08222C000C001C002C00374D5C0E074E2
:1017300017C0E0C082C083C000C00189838882785E
:1017400006742023F0A3D8F97460F0E4D001D0002F
:10175000D083D0827A06E07008BA0602806302174E
:10176000CDB44004A30217D1B42D028071B42E026F
:10177000806CB421028067B42F028062B42302809F
:101780005DBA0002803FB45A0280025030B4300289
:1017900080024029B44102800B5009B43902800410
:1017A000400280192389A0F2A3C082C08389838864
:1017B00082A3A983A882D083D0821A809974FDD392
:1017C0002274FAD32274FED32274F9D322C3740193
:1017D00022C3740022D003D002D001D00022EA2814
:1017E000F8E93400F9AB01AA0078007900A3E060C1
:1017F00024B44004A3021810B430028002401BB489
:10180000390280025014C3943012F0B040BB80DD26
:1018100012181F80BC12181F80B312181F809EE878
:10182000B40F02800250A2234460A903A80289A039
:10183000F222C082C083C000C0F07800E0A308306C
:10184000E0FAE875F00784C5F0700FC5F0E8B41C45
:1018500002800F400DD374FE8005D374FF8000D347
:101860008001C3D0F0D000D083D08222C082C08358
:101870001132400E2582F582E5833400F583E0C302
:007500018A
:101880008001D3D083D08222C000C001C002C00337
:10189000C004C005C006C007740FC0E07419C0E0E2
:1018A0007E02C082C083C000C001C002C003D083DA
:1018B000D082D003D002D001D000121723FF404BBA
:1018C000C082C083C002C003D083D082D003D002C4
:1018D000E82407F8E93400F9121723402EBF01026B
:1018E00080188B838A82E82407F8E93400F91217FC
:1018F000234018B401028002DEECE82406F8E93443
:1019000000F989A0E2D2E0F202190DD322C322D05D
:1019100007D006D005D004D003D002D001D00022D9
:10192000C082C083C000C001C002C003C004C005A3
:10193000C006C00711324073940EFCE5822407F5FF
:1019400082E5833400F583121616405FA903A802CE
:10195000C3E582C39407F582E5839400F5831216EC
:10196000164048E582240EF582E5833400F583A90C
:1019700003A802EC60321CAB83AA8289838882E0D0
:101980006003A380FA7440F0A3A983A8828B838AA2
:10199000821216164015E5822407F582E58334008D
:1019A000F58380CF74FC8003C38001D3D007D006B9
:1019B000D005D004D003D002D001D000D083D08293
:1019C00022C082C083C0F0116C402A30E00630E1B2
:1019D000060219DA0219DA0219F3113240172582C8
:1019E000F582E5833400F583A378FFE008A3B4FF14
:1019F0000780F874FBD38001C3D0F0D083D082225B
:101A0000C0F0116C402C54EF30E00630E106021AB1
:101A100017021A1A021A30B4031611324014258222
:101A2000F582E5833400F583A3E0A3B4FF0780F9D2
:101A300074FBD38001C3D0F022C082C083C0E030E9
:101A4000163B74281214AC121A8474001214ACE5FC
:101A5000822407F582E5833400F583121A84740A20
:101A60001214AC121AF7400A74321214AC121AC0D3
:101A7000800B74321214AC901ABC1214AFD0E0D0A8
:101A800083D08222C082C083C0017906E003121491
:101A9000E0A3D9F8E003540F6014C0E0742D1214D1
:101AA000E0D0E0D4121C1074201214E08006901ACA
:101AB000BC1214AFD001D083D082C32220202000DA
:101AC000C082C08331C1F879FF901B9309E993600C
:101AD00018B500F8E92323901B9E2582F582E58343
:101AE0003400F5831214AF800974301214E0E81248
:101AF0001C10D083D08222C082C083C002C00311D8
:101B00006CAB83AA82F879FF20E013C0E07449121D
:101B100014E0D0E0035477121C10C3021B7A20E1BA
:101B200019540C901BC62582F582E5833400F58399
:101B30001214AF121B92D3021B7A54EFB4030A9013
:101B40001BD61214AFC3021B7AF879FF901BDA0977
:101B5000E993601CB500F8E92323901BE32582F587
:101B600082E5833400F5831214AF121B92D3800AEE
:101B700074301214E0E8121C10D3D003D002D083CA
:101B8000D082222220E708B4200280024001227481
:101B90002E2222060708C3C4CCCDCECFF000435678
:101BA0004A0055564A0053454700544558004C5189
:101BB00050004950200041525000464C58004E45BC
:101BC00054005458540052522000524E5200524574
:101BD0004A0053524A00554920006F2F430F638734
:101BE000AFE3005342450053424D00445343004489
:101BF0004D20005541200046524A005849440054A7
:101C0000535400C0E0E5F0121C10D0E0121C10226A
:101C1000C0E0C412F0A71214E0D0E012F0A7121432
:101C2000E022B40A0280055003121C55B400028061
:101C300024C0E0C000C0F0780075F00A84C0F0084D
:101C400070F7D0F0E5F024301214E0D8F5D0F0D0E1
:101C500000D0E0C322C0E074301214E0D0E0C32210
:101C6000C0D0C082C083C0E0E52A6002152AE549E1
:101C70006012154930130D30170AE5496004C2C4DB
:101C80008002D2C45389F0438901C28C758C4C7593
:101C90008A00D28CD0E0D083D082D0D0325389F069
:101CA000438901C28DC28C758C00758A00D28C224A
:101CB000C000C001C002C0039001401188403090B4
:101CC00001401132F5719001402582F582E583349F
:101CD00000F5837403F0A3057174CCF0A305719033
:101CE0000140780079017A107B013120C38001D353
:101CF000D003D002D001D00022E27D41ADED88D9E1
:101D0000ED503D6786FA1A77A4EF91548147FDF1B3
:101D10003BA2908DB593E2640459CE2D44135D8CA3
:101D2000420CDE003501087D1E88FE74FF38EED1BE
:091D300088F3F06E0E90D0EB79FF
:00000001FF
